:10000000F328820757345834203444346934733425
:1000100070346C34613479342034763430342E3496
:10002000333420340D340A340034E1011E306520AD
:10003000303027202030272028305420083054200A
:10004000013054200C3054200630542008002E205B
:100050000611861086155A2086110800E0006108F6
:100060000F39F038E10083168600831286100615DA
:10007000861506088611861586118039031D3628D7
:10008000061161080F39E1008316860083126008AB
:1000900008002E200611861486155A208611861512
:1000A000E00E5A208611080027208615E00E5A20FF
:1000B000861108000F308605F030600586040800C0
:1000C000A530E200E20B62280800E3006020E30BA9
:1000D00066280800E8000000E80B6C28080083167A
:1000E00005168511A73081000614831285110614A8
:1000F0000030DC20EE00CC20EF000230DC20F100EC
:100100000130DC20F0000330DC20E4000430DC208F
:10011000E5000530DC20E6000630DC20E700393061
:10012000A600A700A800AA00AB00AC002D30A500D7
:100130002030A9000800E9000A30EB000310851107
:10014000031C85156E086A200314E90CEB0B9F282D
:1001500008000D30B22808000A30B228080020300C
:10016000B22808009B286910051E00340930EB00F6
:100170006F086A200310051E0314E90C6E086A203C
:100180000000EB0BBA286908051AC4286914080096
:10019000B320691CC8280800EC00ED010310EC0C2A
:1001A0006C080319DA28ED07EC0C6C080319DA283F
:1001B000ED02CE286D0808007F3983169B001C14C1
:1001C0001A08831208007F3983169B008B131C15B5
:1001D00055309D00AA309D009C141C118B179C1853
:1001E000EF2883120800831207309F006F2015202C
:1001F000A722522106104829851E3822051C3A22C2
:10020000B320691CFC28DF001B3A031909295F0889
:10021000FC28C820DF001B3A031909295F08443A6B
:10022000031933295F08553A03193E295F08563AE6
:10023000031948295F08523A03195C295F08723A8A
:100240000319812A5F08773A031965295F08753A0F
:1002500003199D2A5F08513A0319F3285F08493AA8
:100260000319A722FC28DF01C82083169A008312F5
:100270005F08E320DF0ADF1F3429FC288030B2202A
:10028000DF015F08DC20B220DF0ADF1F4129FC28E4
:10029000DF015F080120003803195129B220DF0A6D
:1002A0004929FC28DF015F080120003803195B2978
:1002B0004920DF0A53290800DF015F088400000895
:1002C000B220DF0A031D5D29FC28061483162130A5
:1002D000A000200884008312C820831684178000A1
:1002E0008413A00A201F7829A01E7829201A7B29B0
:1002F0007106031D6929831280213C220610FC2807
:1003000083162130A000200884008417000884137D
:100310008312A000200865060319A6292008660696
:1003200003190D2A200867060319182A8316A00A44
:10033000201F9E29A01E9E29201AA4298417000888
:1003400084137106031D8329831208001D22A10056
:100350001D22A2001D22A3001D22A40021082502A7
:10036000031CDD29031DDC292118C92926082202C6
:10037000031CDD29031DDC2927082302031CDD29BA
:10038000031DDC2928082402031CDD29031DDC29A8
:10039000DD2922082602031CDD29031DDC29230890
:1003A0002702031CDD29031DDC2924082802031C65
:1003B000DD29031DDC29DD29262229082102031C51
:1003C0000C2A031D0B2A2118F82922082A02031CD3
:1003D0000C2A031D0B2A23082B02031C0C2A031DC5
:1003E0000B2A24082C02031C0C2A031D0B2A0C2A9E
:1003F0002A082202031C0C2A031D0B2A2B082302A5
:10040000031C0C2A031D0B2A2C082402031C0C2A93
:10041000031D0B2A0C2A2F2296291D22AF001D2214
:10042000B0001D22B1001D22B2001D22B30096298A
:100430001D22AD001D22AE0096298316A00A2008B9
:100440008400841700088413831208002108A50083
:100450002208A6002308A7002408A80008002108F5
:10046000A9002208AA002308AB002408AC00080059
:1004700026223C2A2F223C2A803054202108492061
:1004800022084920230849202E30492024084920E9
:1004900043304920203049202F0849203008492086
:1004A00031084920320849202E304920330849209C
:1004B000683049205030492061304920C0305420F4
:1004C0002D0849202E084920253049202030492078
:1004D000290849202A0849202B0849202E30492084
:1004E0002C08492043304920250849202608492066
:1004F000270849202E304920280849204330492028
:10050000080083162130A00020088400841700080A
:1005100084138312B2208316A00A201F932AA01EE0
:10052000932A201A992A8417000884137106031D40
:10053000842A8312A920AC20FC288030B220DF015D
:100540005F08DC20B220DF0ADF1FA02AFC28213050
:100550008400841730308000840A8000840A800080
:10056000840A2F308000840A30308000840A8000A2
:10057000840A8000840A67308000840A303080005A
:10058000840A8000840A8000840A74308000840A0F
:1005900030308000840A8000840A8000840A62303F
:1005A0008000840A30308000840A8000840A800041
:1005B000840A8000840A8000840A68308000840AEB
:1005C00030308000840A8000840A0D308000840A64
:1005D00020308000840A30308000840A8000840A41
:0C05E0008000840A43308000841308006F
:02400E00020DA1
:104200001E002100430074000D00620068000000E1
:0E4210000000000000000000000000000000A0
:00000001FF
